:020000040000FA
:020000001028C6
:100020001F308A0003278A01A1011D20A000A0081B
:10003000031914283920A10A1528210882074334FE
:100040006F346E34673472346134743475346C34A4
:100050006134743469346F346E34733420346634EC
:1000600072346F346D3420344134573443340D349A
:1000700000341F308A00200814278A0108008316E4
:100080008E309F00831281309F007D3023278A01AC
:100090009F149F1849281E3084001F308A001A2799
:0C00A0009E3084001A270D3014274328DE
:00000001FF
